:100000000C94D3060C94F0060C94F0060C94F006B5
:100010000C94F0060C94F0060C94F0060C94F00688
:100020000C94F0060C94F0060C94CE2B0C94A22C9D
:100030000C9440260C94F0060C94F0060C94F006F8
:100040000C94F0060C94F0060C94F0060C94F00658
:100050000C94F0060C94C7260C94F0060C94F00651
:100060000C94F0060C94F0060C94F0060C94F00638
:100070000C94F0060C94F0060C94F0060C94F00628
:100080000C94F0060C94F0060C94F0060C94F00618
:100090000C94F0060C94F0060C94F0060C94F00608
:1000A0000C94F0060C94F0060C94F0062B0014004F
:1000B0001A00080015001700E100040016000700F0
:1000C00009000A00E0001D001B00060019000500E1
:1000D0001C0018000C00120013002A000B000D0079
:1000E0000E000F00330034001100100036003700FE
:1000F00038002800E20022522C002152E743000081
:1001000001001E001F00200021002200010000004D
:1001100000000000000000000100000000000000DE
:1001200000000000230024002500260027004C00CA
:100130005000510052004F00350035024E004B0078
:10014000B600B700B500B4000100010000000100D6
:100150000100000035001E021F02200221022202BF
:10016000010000000000000000000000010000008D
:1001700000000000000000002302240225022D02DE
:1001800031024C00000000000000000031000000BF
:10019000000000000000000000000000010001005D
:1001A0002A00010001000000290020780000000062
:1001B000000000003A003B003C003D003E003F00D4
:1001C00040004100420043004400450000000000A0
:1001D00000000000260227022D0057002E0000001C
:1001E0002F023002A800AA00A90000002F00300052
:1001F00001000100000001000100000044454255DB
:10020000473A2064697361626C65642E0A00444554
:100210004255473A20656E61626C65642E0A000A99
:100220000025303258006C65645F7461736B3A204E
:10023000004F6E6573686F743A2061637469766508
:100240003A2025640A000A0025303862003A20006E
:1002500025303258000A722F632030313233343562
:1002600036370A007267626C696768742074696D5A
:1002700065722064697361626C652E0A0072676240
:100280006C696768742074696D657220656E61625F
:100290006C65642E0A007267626C6967687420730B
:1002A000657420687376205B4E4F454550524F4D24
:1002B0005D3A2025752C25752C25750A007267621C
:1002C0006C696768742073657420687376205B4579
:1002D0004550524F4D5D3A2025752C25752C2575BE
:1002E0000A007267626C69676874207261696E6285
:1002F0006F7720736574206873763A2025642C2507
:10030000642C25642C25750A007267626C69676825
:10031000742064697361626C65205B4E4F45455083
:10032000524F4D5D3A207267626C696768745F6313
:100330006F6E6669672E656E61626C65203D202573
:10034000750A007267626C6967687420646973611A
:10035000626C65205B454550524F4D5D3A20726797
:10036000626C696768745F636F6E6669672E656E3D
:1003700061626C65203D2025750A007267626C69B8
:1003800067687420656E61626C65205B4E4F454501
:1003900050524F4D5D3A207267626C696768745FB6
:1003A000636F6E6669672E656E61626C65203D20C5
:1003B00025750A007267626C6967687420656E61F2
:1003C000626C65205B454550524F4D5D3A20726727
:1003D000626C696768745F636F6E6669672E656ECD
:1003E00061626C65203D2025750A007267626C6948
:1003F00067687420746F67676C65205B4545505271
:100400004F4D5D3A207267626C696768745F636F15
:100410006E6669672E656E61626C65203D2025758C
:100420000A007267626C69676874206D6F6465208A
:100430005B4E4F454550524F4D5D3A2025750A00A1
:100440007267626C69676874206D6F6465205B45D4
:100450004550524F4D5D3A2025750A007267626C17
:10046000696768745F696E6974207267626C696736
:1004700068745F636F6E6669672E6D6F6465203D9B
:1004800020302E2057726974652064656661756C32
:10049000742076616C75657320746F2045455052E9
:1004A0004F4D2E0A007267626C696768745F696EEF
:1004B0006974206565636F6E666967206973206E75
:1004C0006F7420656E61626C65642E0A00726762EB
:1004D0006C696768745F696E6974207374617274A3
:1004E000210A007267626C696768745F696E69747B
:1004F0002063616C6C65642E0A007267626C6967C8
:1005000068745F636F6E6669672E737065656420DB
:100510003D2025640A007267626C696768745F63D6
:100520006F6E6669672E76616C203D2025640A0037
:100530007267626C696768745F636F6E6669672E65
:10054000736174203D2025640A007267626C6967DC
:1005500068745F636F6E6669672E687565203D20FD
:1005600025640A007267686C696768745F636F6E00
:100570006669672E6D6F6465203D2025640A0072F0
:1005800067626C696768745F636F6E6669672E7611
:10059000656C6F63696B6579203D2025640A007284
:1005A00067626C696768745F636F6E6669672E6502
:1005B0006E61626C65203D2025640A007267626C82
:1005C000696768745F636F6E66696720454550525E
:1005D0004F4D3A0A001E0F0500047F3F1F6432147E
:1005E000643214783C1E1E140A052223252628296D
:1005F0002A2C2D2F3032333536383A3B3D3E40429F
:10060000434547494A4C4E5051535557595A5C5EE1
:100610006062646668696B6D6F71737577797B7DF5
:100620007F81838587898A8C8E90929496989A9CF4
:100630009E9FA1A3A5A7A8AAACAEAFB1B3B4B6B80C
:10064000B9BBBCBEBFC1C2C3C5C6C7C9CACBCCCD6E
:10065000CED0D1D2D2D3D4D5D6D7D7D8D9D9DADA49
:10066000DBDBDBDCDCDCDCDCDDDDDDDDDCDCDCDCC9
:10067000DCDBDBDBDADAD9D9D8D7D7D6D5D4D3D2FD
:10068000D2D1D0CECDCCCBCAC9C7C6C5C3C2C1BFDB
:10069000BEBCBBB9B8B6B4B3B1AFAEACAAA8A7A53F
:1006A000A3A19F9E9C9A98969492908E8C8A8987FB
:1006B0008583817F7D7B79777573716F6D6B6968D9
:1006C000666462605E5C5A5957555351504E4C4AAD
:1006D0004947454342403E3D3B3A38363533323058
:1006E0002F2D2C2A292826252322FFAA7F554000BA
:1006F00001010101010101010102020202020202E3
:1007000002020303030303030303040404040404B5
:10071000040505050505060606060607070707077B
:1007200008080808090909090A0A0A0B0B0B0C0C2E
:100730000C0D0D0D0E0E0E0F0F0F101011111112CA
:100740001213131414151516161717181819191A49
:100750001A1B1B1C1D1D1E1E1F20202122222324AC
:1007600024252626272829292A2B2C2D2D2E2F30EB
:10077000313232333435363738393A3B3C3D3E3FFF
:10078000404142434445464748494A4C4D4E4F50EC
:10079000515354555658595A5B5D5E5F61626465AA
:1007A0006668696B6C6D6F7072737577787A7B7D34
:1007B0007E8082838587888A8C8E8F919395969888
:1007C0009A9C9EA0A2A3A5A7A9ABADAFB1B3B5B7A4
:1007D000BABCBEC0C2C4C6C9CBCDCFD1D4D6D8DB7B
:1007E000DDDFE2E4E7E9EBEEF0F3F5F8FAFDFF3FD9
:1007F00000433E20004C25640A000A092D20537452
:1008000061747573202D0A686F73745F6B6579620C
:100810006F6172645F6C65647328293A20253032F9
:10082000580A6B6579626F6172645F70726F746F82
:10083000636F6C3A20253032580A6B6579626F61BC
:1008400072645F69646C653A20253032580A7469B5
:100850006D65725F72656164333228293A202530F4
:10086000386C580A002573000A092D20436F6E73F7
:100870006F6C65202D0A4553432F713A09717569D4
:10088000740A000A092D204D61676963202D0A440E
:100890003A094465627567204D6573736167652029
:1008A000546F67676C650A583A094D6174726978CC
:1008B000204465627567204D6F646520546F6767DB
:1008C0006C65202D2053686F77206B657970726599
:1008D0007373657320696E206D6174726978206727
:1008E0007269640A4B3A094B6579626F61726420E0
:1008F000446562756720546F67676C65202D2053CF
:10090000686F77206B65797072657373207265709C
:100910006F72740A4D3A094465627567204D6F75B0
:10092000736520546F67676C650A563A095665729D
:1009300073696F6E0A533A095374617475730A438D
:100940003A09416374697661746520436F6E736F11
:100950006C65204D6F64650A46312D4631303A0989
:1009600053776974636820746F204C6179657220D5
:10097000302D392028463130203D204C30290A3096
:100980002D393A0953776974636820746F204C617C
:1009900079657220302D390A47524156453A09533C
:1009A000776974636820746F204C617965722030B8
:1009B0002028616C7465726E617465290A423A0977
:1009C0004A756D7020746F20426F6F746C6F616434
:1009D00065720A4553433A094A756D7020746F2059
:1009E000426F6F746C6F616465722028616C74650E
:1009F000726E617465290A453A095072696E7420F5
:100A0000454550524F4D2053657474696E67730AA3
:100A10004241434B53504143453A09436C6561722F
:100A200020454550524F4D0A006B65796D61705FEE
:100A3000636F6E6669672E7261773A20253032588F
:100A40000A2E737761705F636F6E74726F6C5F6391
:100A50006170736C6F636B3A2025750A2E63617049
:100A6000736C6F636B5F746F5F636F6E74726F6CC8
:100A70003A2025750A2E737761705F6C63746C5F22
:100A80006C6775693A2025750A2E737761705F72FD
:100A900063746C5F726775693A2025750A2E7377E7
:100AA00061705F6C616C745F6C6775693A20257565
:100AB0000A2E737761705F72616C745F726775691B
:100AC0003A2025750A2E6E6F5F6775693A20257585
:100AD0000A2E737761705F67726176655F65736315
:100AE0003A2025750A2E737761705F6261636B73BC
:100AF0006C6173685F6261636B73706163653A20F8
:100B000025750A2E6E6B726F3A2025750A2E737743
:100B100061705F6573636170655F636170736C6F53
:100B2000636B3A2025750A0064656275675F636FC1
:100B30006E6669672E7261773A20253032580A2E28
:100B4000656E61626C653A2025750A2E6D6174725E
:100B500069783A2025750A2E6B6579626F61726437
:100B60003A2025750A2E6D6F7573653A2025750A32
:100B7000006565636F6E6669673A0A6465666175EC
:100B80006C745F6C617965723A2025750A003F00CC
:100B90000A6D6F7573653A206F66660A000A6D6F9D
:100BA0007573653A206F6E0A000A6B6579626F6132
:100BB00072643A206F66660A000A6B6579626F613B
:100BC00072643A206F6E0A000A6D61747269783A35
:100BD000206F66660A000A6D61747269783A206F48
:100BE0006E0A000A64656275673A206F66660A00DD
:100BF0000A64656275673A206F6E0A000A0A4A75D0
:100C00006D70696E6720746F20626F6F746C6F61B6
:100C10006465722E2E2E2000433E2000436C6561D9
:100C200072696E6720454550524F4D0A000A0025F3
:100C300030325820006B6579626F6172645F726553
:100C4000706F72743A2025303258207C2000737502
:100C50007370656E64696E67206B6579626F61722F
:100C6000640D0A005B575D005B535D005B525D00E5
:100C70005B445D005B435D00140372006500760019
:100C8000690075006E0067003400310000000C033D
:100C90006700740069007000730000000403090419
:100CA00009025B00030100A0FA090400000103012E
:100CB00001000921110100012244000705810308F8
:100CC00000010904010001030000000921110100D5
:100CD00001223200070582032000010904020002FC
:100CE00003000000092111010001222200070583F1
:100CF0000320000107050303200001120100020088
:100D00000000080778CBDC0100010200010631FF7A
:100D10000974A1010975150026FF00952075088149
:100D2000020976150026FF00952075089102C0057E
:100D3000010980A101850319012AB700150126B711
:100D400000950175108100C0050C0901A101850401
:100D500019012AA002150126A00295017510810033
:100D6000C005010906A101050719E029E7150025BD
:100D70000195087501810295017508810105071922
:100D80000029FF150026FF0095067508810005085B
:100D90001901290515002501950575019102950197
:100DA00075039101C00011241FBECFEFDAE0DEBF52
:100DB000CDBF12E0A0E0B1E0E8E3F1E602C00590AB
:100DC0000D92A239B107D9F723E0A2E9B2E001C040
:100DD0001D92AA3CB207E1F70E9489170C94463095
:100DE0000C940000FF93EF93E0919202F091930234
:100DF000309709F00995EF91FF910895FC018591D5
:100E0000803011F0EFDFFBCF0895FF27E0E230E202
:100E100047FF0CC0419597FF09C0EDE260957095C2
:100E200080959095611D711D811D911D27FF02C048
:100E3000219530E350E2AA27660F771F881F991F7C
:100E4000AA1FA41710F0A41B63955A95A9F7AA30FE
:100E500008F0A95FA05DAF93F39561157105810559
:100E6000910541F7ED3211F4EF93F395F21718F471
:100E70003F93F395FBCF8F91B5DFFA95E1F7089596
:100E8000E991F9918591803021F0853219F0AADF3E
:100E9000F9CF089520E0E89455915532C1F35033CD
:100EA00011F4689455915A3348F4505390F3220F3B
:100EB000022E220F220F200D250FF4CF0EF42195C4
:100EC00089919991533619F3533729F1533559F1D3
:100ED000BC0188279927E8945C3621F4899199917F
:100EE00068945591543639F446EF7EF077FF0DC083
:100EF0008FEF9FEF0AC055374AE039F0583540E18F
:100F000021F0523642E009F00895FF93EF937DDF20
:100F1000EF91FF91B7CFFF93EF93FC018191803068
:100F2000B9F360DFFBCFFF93EF9368DFF1CFDF937F
:100F3000CF93CDB7DEB72596A3DFCF91DF9108958C
:100F40008430B8F46730A8F4463098F450E096E066
:100F5000699F400D511D1124FA019AE2899FE00D0D
:100F6000F11D1124EE0FFF1FE455FF4F8591949161
:100F7000089581E090E008950E94A007089581E01F
:100F800008950E94BF07089581E008950E94BF0759
:100F900008950E94C607089508950E94CC070895F9
:100FA000A6E0B0E0E6EDF7E00C94F22E49835A8318
:100FB0009E833091990289819A8131111AC03E81B4
:100FC000332399F0222389F00E94110E182F682FE5
:100FD00089819A810E94ED0D69817A81812F0E9419
:100FE000E3142696E3E00C940E2F0E94FF0D182FB9
:100FF000F3CF0E94110E69817A81F1CFFC01262F77
:101000004081518162817381848195810E94D007E2
:101010000895CF93DF93EC0161E00E94FE07BE01CB
:101020000E94C107DF91CF910895CF93DF93EC0128
:1010300060E00E94FE07BE010E94CD07DF91CF91C4
:10104000089581E008950E9421080895CF93C82F44
:101050000E94C20C8C2F0E9423082FEF84E39CE097
:10106000215080409040E1F700C00000CF910895EA
:1010700081E00E9426080E94EB26089580E00E94ED
:1010800026080E94FC2608950F931F93CF93DF93A9
:101090008C0161E00E94FE07EC01F801858181115D
:1010A0000E94B120B801CE010E94C907811106C07B
:1010B00080E0DF91CF911F910F910895B801CE018B
:1010C0000E94A3248823A1F3B801CE010E946323C8
:1010D000882371F3B801CE010E943923882341F39C
:1010E000B801CE010E94D020882311F3F801858138
:1010F000882369F0C330FCE7DF0781F160F4C13079
:10110000ECE7DE0769F1C0F4C115DC4791F0C801D6
:101110000E94C407CECFCB35ECE7DE0739F1CC35E2
:10112000FCE7DF0701F1CA35DC4789F70E943B1273
:10113000EECF0E943808BCCF90911D03892F8E7F7F
:1011400090FF816080931D0380FF05C08EE092E0D8
:101150000E94FE06ADCF8CEF91E0FACF0E944312C1
:101160000E943E08A5CF0E943112D1CF0E943F12AB
:10117000CECF0E941D260E94FC080E9401200895E7
:101180000E9400090E94921F0E94222608958295C3
:1011900090E09C01220F331F220F331F2C7C95956A
:1011A0008795959587958373282B30E0C901880F23
:1011B000991F8A7A359527952575822B089508956C
:1011C00081E008950895CF93DF93D82F0E94E0081F
:1011D000C82F882319F08D2F0E94E2088C2FDF91F1
:1011E000CF9108950895CF93C82F0E94DF088C2FC8
:1011F0000E94E308CF91089580E00E94F3080895CB
:101200000E94EC240E94F3080895CF930E94EC24DE
:10121000C82F809194028C1789F1C09394020E9488
:10122000AC266093950270939602809397029093F8
:10123000980280911D0382FF1EC080FF1CC086E2C1
:1012400092E00E94FE0680911D0380FF14C01F9251
:10125000CF9381E292E09F938F930E9497078091B2
:101260001D030F900F900F900F9080FF04C08FE12F
:1012700092E00E94FE068C2F0E94F308CF91089501
:10128000ADE0B0E0E6E4F9E00C94F32E488759872E
:101290006A877B878C879D8791110E945E111F82D0
:1012A00086E0FE013896DE01119601900D928A9536
:1012B000E1F78D8181110DC029813A814B815C81DB
:1012C0006D817E818F810E94A8102D96E2E00C94A2
:1012D0000F2FCE0101960E9409088111EDCFF5CFA5
:1012E000FC012481213021F4808191810E94430EF0
:1012F0000895CF93C82F8823C9F08238C9F40E947B
:10130000F92481FD13C089E30E94E0250E94CD11DC
:101310002FEF87EE93E0215080409040E1F700C02E
:10132000000089E30E94E8250E94CD11CF91089525
:101330008338A1F40E94F92480FDF8CF83E50E9450
:10134000E0250E94CD112FEF81EE94E021508040E6
:101350009040E1F700C0000083E5E4CF8438A1F4B9
:101360000E94F92482FDE2CF87E40E94E0250E94DA
:10137000CD112FEF81EE94E0215080409040E1F7B5
:1013800000C0000087E4CECF8CEF8C0F813A98F438
:101390008C2F0E94F6228111C9CF8C2F0E94A52587
:1013A000882329F08C2F0E94E8250E94CD118C2FD4
:1013B0000E94E025B9CF80E28C0F883048F4C770D6
:1013C00081E001C0880FCA95EAF70E944111ACCFB5
:1013D000EBE5EC0FE33040F4F0E0E65AFE4F80819D
:1013E00090E00E944625A2CFC85ACB3108F09ECF8C
:1013F000EC2FF0E0EE0FFF1FEC5DFE4F808191813E
:101400000E946B2593CF882309F44DC0823879F46C
:101410000E94F92481FF47C089E30E94E0250E94D1
:10142000CD1189E30E94E8250E94CD1108958338EB
:1014300059F40E94F92480FF36C083E50E94E0251C
:101440000E94CD1183E5EECF843859F40E94F9242F
:1014500082FF29C087E40E94E0250E94CD1187E425
:10146000E1CF9CEF980F913AE8F290E2980F983014
:1014700050F4877091E001C0990F8A95EAF7892F9F
:101480000E944711D1CF9BE5980F933028F490E04C
:1014900080E00E9446250895885A8B3120F490E020
:1014A00080E00E946B2508951F93CF93DF93182F40
:1014B000EB010E947909209739F4812F0E94030AD9
:1014C000DF91CF911F9108958FE99FE00197F1F788
:1014D00000C000002197EFCF70E060E0893311F485
:1014E00060E570E00E94540A0895882321F00E946C
:1014F00041110E94CD110895882321F00E944711C7
:101500000E94CD110895B0E0A0E0E9E8FAE00C9463
:10151000EC2E6C01D62FC72FFC0115810681029598
:101520000F700E943711E82E8823F9F0E12E112365
:10153000E1F08C2F807F803461F080E28D0F883065
:1015400008F18C2F807E803221F4D230D8F0002335
:10155000C9F08091810382FF15C082E00E94F211E0
:101560000E94371191E0E82EE926BC2EB2949FE04C
:10157000B922FBE0FB15B8F1EB2DF0E0E85BFF4C86
:101580000C94AC2EE12CF1CF0C2F0F70C07F11F01A
:101590000295007F112399F0002359F080E28D0F0E
:1015A000883010F0D11107C0802F0E9441110E9495
:1015B000CD118D2F5AC0802F0E945111F8CF8D2F41
:1015C0000E94030A002379F080E28D0F883010F02A
:1015D000D11104C0802F0E94471103C0802F0E94A8
:1015E00057110E94CD11EB2DE850FF0B349720F4DA
:1015F0000E94EC240E94F308EE2089F00E9433112F
:1016000080FD0DC0F60115820E942D110E944B0D28
:10161000C6010E948D0C0E942D110E945B0DCDB75A
:10162000DEB7E9E00C94082F2C2F2F70F22EC07F2C
:10163000C03219F0F29480EFF822DD2341F0D1306E
:10164000D1F1112309F444C00023F1F0B2CF80910D
:10165000810382FD15C0112359F0FF2029F08F2D41
:101660000E9441110E94CD1180E00E947909BBCFF8
:1016700080E00E94030AFF2009F4B5CF8F2DABCF85
:10168000112369F0011104C08F2D0E94750AABCFA0
:10169000013009F0A8CF8F2D0E947511A4CF011140
:1016A000A2CF8F2D0E947C0A8F2D0E9481118F2D39
:1016B0000E94651198CF112321F0063008F093CFD6
:1016C000E3CF053008F08FCF8F2D0E947C0A8BCF9F
:1016D0000023D1F3D93349F43FEF87EE93E0315043
:1016E00080409040E1F700C000008D2F0E94030A67
:1016F0007ACF8C2F86958695837069F0813009F0BA
:1017000072CF8D2F9C2F9370111102C080E090E05A
:101710000E946B2568CF8D2F9C2F9370111102C0F2
:1017200080E090E00E9446255ECF8C2F8370A1F56B
:10173000111159CF4D2F429546954770440F440FD4
:101740002D2F2F7030E0042E02C0220F331F0A9479
:10175000E2F790E080E0D4FF09C08FE090E002C0A3
:10176000880F991F4A95E2F780959095C695C69582
:10177000C370822B932BC23049F058F4C13019F05A
:101780000E941B0D30CF0E94120D2DCF0E94240D00
:101790002ACF0E940F0D27CF8695112311F08C2F91
:1017A0008170882309F41FCF4D2F429546954770CD
:1017B000440F440F2D2F2F7030E0042E02C0220F53
:1017C000331F0A94E2F790E080E0D4FF09C08FE075
:1017D00090E002C0880F991F4A95E2F78095909596
:1017E000C695C695C370822B932BC23049F058F42E
:1017F000C13019F00E94860DF6CE0E947D0DF3CE09
:101800000E948F0DF0CE0E94330DEDCECF701123CC
:1018100029F08C2F0E944B0D8D2F37CF8D2F0E94DA
:101820007C0A8C2F0E945B0DDECED23F41F160F42A
:10183000D03FB9F0D13F81F0112309F446C0011126
:10184000B8CE8C2F8F711FC0D33F01F1D43FA1F7C9
:101850008091810382FD24C08C2F8F71112311F39D
:1018600012C0112341F0053008F0BDCE8C2F8F71CE
:101870000E946D0DB8CE063008F0B5CEF7CF8C2F94
:101880008F711111CFCF0E944B0DADCE112329F0D6
:101890008C2F8F710E943F0DA6CE0E943A0DA3CED1
:1018A000112349F0CF718C2F0E944B0D63E08C2FD8
:1018B0000E94D41198CE81E00E94F211023008F407
:1018C00092CE82E00E94F2118ECE002359F0D933DD
:1018D00009F00BCFEFEFF7EE23E0E150F0402040AE
:1018E000E1F701CF8C2F8F719DCF0F931F93CF9373
:1018F000DF93EC01688179818D810E944E0E8C010D
:101900000E94980D0E940E0DB801CE010E94830A1C
:10191000DF91CF911F910F910895CF93DF93EC0149
:101920008C81882399F0CE010E944408811111C056
:101930000E943711882351F08D81882339F08091DE
:10194000810382FF03C082E00E94F211DF91CF91F8
:101950000895CE010E94750CCE010E941508F6CFA5
:1019600090E080E00E94462590E080E00E946B2598
:101970000E945E110E94CD1108950E94F0250E94E0
:10198000B00C08950E944E110E94BD0C08959295CE
:101990009F70963091F058F4925F9F70923058F497
:1019A000803F19F030F4883E30F481E008959A5F6A
:1019B000F4CF843FD1F380E00895883EB0F3813FB7
:1019C000D1F7F3CFFC012481222339F0808191816A
:1019D0000E94430E0E94C70C089580E00895A6E07F
:1019E000B0E0E5EFFCE00C94F32E2696E2E00C94D8
:1019F0000F2FA7E0B0E0EFEFFCE00C94F32E27965A
:101A0000E2E00C940F2F08950E94030D08950E94A8
:101A1000040D9093B5028093B402089508950E9436
:101A2000070D08952091B4023091B502822B932BBB
:101A30000E94070D08952091B4023091B5028223CF
:101A400093230E94070D08952091B4023091B502AE
:101A5000822793270E94070D08950E94030D089581
:101A60000E942D0D08950E94300D9093B302809333
:101A7000B202089590E080E00E94330D089521E0C5
:101A800030E0A90102C0440F551F8A95E2F7CA0150
:101A90000E94330D089521E030E002C0220F331F71
:101AA0008A95E2F78091B2029091B302822B932B38
:101AB0000E94330D089521E030E002C0220F331F51
:101AC0008A95E2F7209530958091B2029091B30209
:101AD000822393230E94330D089521E030E002C059
:101AE000220F331F8A95E2F78091B2029091B302E0
:101AF000822793270E94330D08952091B2023091DE
:101B0000B302822B932B0E94330D08952091B202D1
:101B10003091B302822393230E94330D08952091C4
:101B2000B2023091B302822793270E94330D0895A9
:101B30000895262F277091E001C0990F2A95EAF7A2
:101B400023E0769567952A95E1F7660F771F660F74
:101B5000771FFA01E60FF71F50E040E0682F70E0B2
:101B60008191DF0111979B01042E02C036952795C4
:101B70000A94E2F7217021952827292328272C93FE
:101B80004F5F5F4F4430510559F70895A82FA77054
:101B900023E0969587952A95E1F7880F991F880F7E
:101BA000991FFB01E80FF91F50E040E080E0219110
:101BB00030E00A2E02C0369527950A94E2F721708C
:101BC0003327042E01C0220F0A94EAF7822B4F5FBD
:101BD0005F4F4430510559F70895262F973070F420
:101BE000863060F4682F70E086E0989F600D711D6C
:101BF00011244AE952E0822F0E94990D0895292F5D
:101C0000973068F4863058F490E06AE972E036E084
:101C1000239F800D911D11240E94C60D089580E020
:101C20000895B0E0A0E0E7E1FEE00C94EC2E7C012A
:101C30000091B2021091B3028091B4029091B5026A
:101C4000082B192BCFE0D0E0CC24C394D12CBC2E90
:101C5000C6010C2E02C0880F991F0A94E2F7802358
:101C60009123892B49F4219790F7B12C8B2DCDB777
:101C7000DEB7E9E00C94082FB7018C2F0E94EF1417
:101C8000019789F3F3CFCF93DF93EC010E94110EFC
:101C9000BE010E94EF14DF91CF9108951F93CF935F
:101CA000DF93EB0190919902992339F0CB010E94C7
:101CB000430EDF91CF911F910895882369F0CB01E6
:101CC0000E94110E182F682FCE010E94ED0DBE014B
:101CD000812F0E94EF14EDCFCB010E94FF0D182F32
:101CE000F6CF1F93CF93DF93C091B60217E0809198
:101CF000B7028C1304C0DF91CF911F910895D0E0FB
:101D00001C9FF0011D9FF00D1124E854FD4F208110
:101D10003181428153816481758186810E94F90CF1
:101D20002196C770E4CF2091F0023091F1024091EA
:101D3000F2025091F3026091F4027091F5028091E9
:101D4000F6020E94F90C0895CF93DF938091F6027A
:101D5000807F09F04DC08091F502882309F448C0C6
:101D6000E091B6025091B702C091F102D091F00219
:101D70006091F2027091F30247E05E17C9F18E2F75
:101D800090E0E49FF0011124E854FD4F24812223C8
:101D900091F1489FF001499FF00D1124DF01A854F3
:101DA000BD4F11962C9111972C1325C02C912D13FA
:101DB00022C015962C91159721111DC012962D91B8
:101DC0003C91261B370B283C3105A8F48091F60284
:101DD0008F7080618093F602E254FD4F80818F7096
:101DE0008061808380EF92E00E948D0C0E94710ED2
:101DF000DF91CF910895FC013196E770BECF482F57
:101E00002091B6029091B70257E0291302C080E0FA
:101E1000089530E0529FF001539FF00D1124E854D3
:101E2000FD4F8181681306C08081481303C08581FE
:101E30008111EECF2F5F3F4F2770E7CFA4E1B0E0D5
:101E4000E4E2FFE00C94E92E8C0186E0F801DE016B
:101E50001F9601900D928A95E1F7F8018481E58043
:101E600090EFA92E92E0B92E9091F40291111FC02B
:101E70008823D1F0EE20A9F0C8010E94E20CF82ED0
:101E8000882379F087E0F801D50101900D928A95B9
:101E9000E1F7C5010E9470090E94A40E0E94930EF2
:101EA0005FC0C8010E948D0CFF24F39459C0C0800C
:101EB000D18082809380F090F5022091F2023091DF
:101EC000F302A401421B530BFF2009F4F9C0483C64
:101ED000510508F0A7C0882309F442C09091F1028F
:101EE0008091F602282F207F09F05CC09D1116C05A
:101EF0009091F002C91212C0E1104EC08F70806143
:101F00008093F6020E94930E80EF92E00E948D0C67
:101F10008091F602F8018683F12C22C0E1103CC0CA
:101F20006D2D8C2D0E94FF0E6D2D8C2D0E94FF0EAD
:101F3000E82E8111F1CFCF86D88A8F8598890E94AB
:101F4000430E292F22952F70243078F49F70223071
:101F5000A8F09923B9F0F8019681907F99F4FE2CAE
:101F60008F2D6496ECE00C94052F2A5F2F702230A1
:101F700068F0C8010E948D0CEF2CF1CF992311F06D
:101F8000882369F3805E883050F3F3CF803F38F3C5
:101F9000815F833070F7E3CF8091F6028160809398
:101FA000F602BACF9D1113C09091F002C9120FC072
:101FB000E1100DC08683C8010E948D0C87E0F801F6
:101FC000A0EFB2E001900D928A95E1F767CFC801CA
:101FD0000E94E20C882309F464CFEE2009F461CF5B
:101FE0008091F602803288F02091F0023091F10267
:101FF000398728879B868A869091F4029C871D8664
:102000008E87CE0108960E948D0C87E0F801A0EF24
:10201000B2E001900D928A95E1F70E94A40E0E9411
:10202000930E42CF9091F602292F207FA1F4682DC4
:102030009A8A898AA6017A899E2D0E94EF0C80EFE8
:1020400092E00E948D0C87E0F50111928A95E9F7E4
:102050000E94930E61CF882309F482CF8091F10210
:102060008D1110C08091F002C8120CC0E1100AC09E
:102070009683C8010E948D0C87E0F50111928A9524
:10208000E9F76ECFC8010E94E20C882309F409CF5A
:10209000EE2009F406CF8091F602803208F4B5CF25
:1020A0002091F0023091F1023A8329839C828B8245
:1020B0009091F4029D831E828F83CE010196A3CF5F
:1020C000483C5105B8F5882309F4EECEFE2CEE20ED
:1020D00009F4E7CE8091F1028D111EC08091F002CB
:1020E000C8121AC08091F60280FD0DC0982F907F13
:1020F00051F08683903F09F45ECF982F907F905FD8
:102100008F70892B57CF87E0F801A0EFB2E00190E4
:102110000D928A95E1F724CFC8010E94E20C81114B
:1021200074CF8091F60281608093F602C8010E940C
:102130008D0C16CF682D9A8A898AA6017A899E2DE0
:102140000E94EF0C87E0F50111928A95E9F7A6CE7F
:10215000AEE0B0E0EEEAF0E10C94F22E2887398789
:102160004A875B876C877D878E87CE0108960E94A1
:102170001E0F8823B1F06C85662341F028853985D0
:102180004A855B857D858E850E94F90C17E08091DC
:10219000B6029091B70289133DC02E96E3E00C94ED
:1021A0000E2F87E0FE013896DE01119601900D9208
:1021B0008A95E1F78C85882349F32091B70230E0B6
:1021C000C9010196877099274091B60248171906F0
:1021D00099F097E0929FD001939FB00D1124A854DD
:1021E000BD4FFE01319601900D929A95E1F78093D3
:1021F000B7020E94710ECACF0E94C20C1092B702A1
:102200001092B60287E0E0EFF2E0DF011D928A95BE
:10221000E9F7BCCF819FC001112488549D4F0E94D3
:102220001E0F882309F4B9CFE091B6021E9FF0017A
:102230001124E854FD4F2081318142815381648112
:10224000758186810E94F90C8091B60290E001961A
:10225000877099278093B6029ACF8091FF02869566
:102260008695869508958091FF02877008959091D4
:10227000FF02977081E009F480E0089580910B03DC
:10228000089590910B03892B80930B0308958095FB
:1022900090910B03982390930B03089510920B03D6
:1022A000089590910A03892B80930A0308958095DD
:1022B00090910A03982390930A03089510920A03B9
:1022C000089508950E946111089590910003292FA7
:1022D000282331F080958923809300030E946211A6
:1022E000089508950E947111089590910103292F76
:1022F0002823281729F0982B909301030E9472112C
:10230000089590910103292F282331F08095892386
:10231000809301030E947211089580910103882324
:1023200029F01092010380E00E94721108950F932A
:102330001F93CF93DF930091040110910501C09189
:102340000B0380910A03C82B80910103882331F08D
:10235000C82B0E94902581110E948D11F801C08325
:10236000C0910401D091050148E050E067EF72E0B0
:10237000CE010E94B92F892B59F088E0FE01A7EF0A
:10238000B2E001900D928A95E1F7CE010E94FC2403
:10239000DF91CF911F910F9108950E949711089599
:1023A00008950E94D01108959091810392FF11C069
:1023B00098E0899F90011124622B6093FF020E9494
:1023C0004B0D8091FF028695869586950E94D111CE
:1023D00008950E944B0D08951092FF0280E00E9424
:1023E000D11108959091FF02809589238093FF0277
:1023F000282F277069F4891759F09091810392FF73
:1024000007C08695869586950E945B0D0E94EC110B
:102410000895CF93C82F8091810382FB992790F96B
:102420009C17E9F0C0FB82F98093810380918003BF
:10243000909181030E94641282E00E94F2118091C7
:102440001D0380FF0CC01F92CF9381E392E09F9306
:102450008F930E9497070F900F900F900F90CF913E
:1024600008958091810382FB882780F991E0892774
:102470000E940912089581E00E940912089580E0E7
:102480000E94091208956FEF7FEF90E080E00E94B4
:102490001130089590E080E00E94DD2F21E0863E1B
:1024A0009E4F09F020E0822F089582E090E00E9484
:1024B000CF2F089583E090E00E94CF2F089584E00D
:1024C00090E00E94DD2F0895BC0184E090E00E941E
:1024D00011300895AB01BC018FE090E00E940530FF
:1024E0000895AB01BC0183E190E00E94053008959E
:1024F00060E070E0CB010E947112089560E070E02E
:10250000CB010E946A120E9478120895A8E0B0E000
:10251000ECE8F2E10C94F32E66EE7EEF90E080E0C2
:102520000E94113060E082E090E00E94F32F81E091
:1025300090E09093B5028093B40261E083E090E074
:102540000E94F32F60E074E184E090E00E9411307B
:1025500060E086E090E00E94F32F6FEF87E090E06C
:102560000E94F32F40E050E0BA0188E090E00E9422
:10257000053060E084E290E00E94F32F60E087E1A4
:1025800090E00E94F32F60E08CE090E00E94F32F37
:1025900060E08DE090E00E94F32F19821A821B8286
:1025A0001C821D821E821F82188648E050E068E16E
:1025B00070E0CE0101960E94E32F40E050E0BA01A6
:1025C00080E290E00E9405300E947E122896E2E0B0
:1025D0000C940F2F0E9486120895682F8EE090E0D1
:1025E0000E94F32F0895A6E0B0E0E9EFF2E10C9429
:1025F000F12E0E94A0268C0180910C0390910D0376
:102600008017910781F019821A820E94A026682FF4
:1026100049815A81792F80E090E00E94400910930F
:102620000D0300930C032696E4E00C940D2F0E94FA
:10263000AC266093190370931A0380931B03909345
:102640001C036093150370931603809317039093F4
:1026500018030895089508950E942A13089508956F
:102660000E942F1308958CE998E20E9496170E9409
:102670002B130E942C13089581E008950E943C13AF
:1026800008950E943C130895089508950E944413EC
:102690000E94451308950E94E6150E94F2080895CD
:1026A0000E9497260E94F0160E944B130E94FF1E64
:1026B0000E9430130895A6E0B0E0E1E6F3E10C9447
:1026C000EA2E0E943E1381110AC00E94F3120E945A
:1026D000B2200E9405092696EBE00C94062F0E947A
:1026E00006178EE0A82E83E0B82E750110E0F701E2
:1026F00001917F01812F0E940C161F5F173009F492
:1027000041C00817A1F380911D0381FD0E9412169C
:102710000E944113C82E10E099249394812F0E94A7
:102720000C16082FF50181915F01081729F1F12C92
:10273000EE24E394D02ED8268D2D8E21A9F0CC2026
:1027400099F0F9821A830E94A0269C838B839D8234
:1027500091E0802F8E2109F490E049815A816B81AC
:102760007C818D810E944009F394EE0CF6E0FF120B
:10277000E3CFF501319700831F5F173079F60E9490
:102780001713A5CF0813BFCFA0CF1F93CF93DF930D
:102790000E94F414EC01C11580E5D807F0F5C115CD
:1027A00080E4D80708F09CC0C03ED10520F5CD3CA0
:1027B000D10508F082C0C83AD10578F4C53AD105F0
:1027C00008F073C0C130D10519F1209709F1C43068
:1027D000D105F0F4D0E0C0E01BC0C33CD105D0F778
:1027E000C85AD0E0CC0FDD1FC35ADE4F0990D88104
:1027F000C02DD4640DC0C11580E2D80708F0D1C047
:10280000C11581E0D80708F05AC0C83ED10510F7BD
:10281000CE01DF91CF911F910895C03682E5D80790
:1028200018F5C03482E5D80708F06BC0C03282E5E5
:10283000D80708F05FC0C11582E5D80708F497C033
:102840002C2F2695269580E2289F900111248C2F0D
:102850008370C1E0D0E002C0CC0FDD1F8A95E2F7A3
:10286000C22BD32BDD68D4CFC03A82E5D80760F401
:10287000C03882E5D80708F459C0CF71D0E0DC2F0A
:10288000CC27C46FD06AC4CFC03C82E5D80708F417
:1028900062C0C03E82E5D80708F09CCFDC2FCC2771
:1028A000CC27DF71C06FD06AB3CFC55AD0E0CD5608
:1028B000DE4FC881D0E0D064ABCFD065A9CF8D2FDB
:1028C0000E949615182FCE0199270E94F414C12F4B
:1028D000D0E0DC2FCC27CC27DF71C82BD92B98CFA9
:1028E000CE0199270E94F414CC27DF70C82BD92B76
:1028F000D06A8ECFCF71D0E0DC2FCC27C16FD06AE9
:1029000087CF2C2F26952695277080E2289F90014F
:1029100011248C2F8370C1E0D0E002C0CC0FDD1FEA
:102920008A95E2F7C22BD32BDC6872CF2C2F269529
:102930002695277080E2289F900111248C2F8370A8
:10294000C1E0D0E002C0CC0FDD1F8A95E2F7C22BB8
:10295000D32BDA685DCF8C2F8F710E949615C82F0C
:10296000D0E0DC2FCC27CC27DF71D06251CF8C2F69
:102970008F710E94961555E0D695C7955A95E1F747
:10298000CF70D0E0DC2FCC27282F30E084FF05C0AB
:1029900044E0220F331F4A95E1F7C22BD32BD069B5
:1029A00037CF8D2F8F710E949615182FCE01992742
:1029B0000E94F414C12FD0E0DC2FCC27CC27DF718C
:1029C000C82BD92BD2CF462F773030F4663020F485
:1029D000672F0E94BC07089590E080E008950E9450
:1029E000E3140E94C513089582389105B9F1B0F43B
:1029F0008133910509F47DC048F48932910509F4C9
:102A00006DC08A32910509F47BC008958533910524
:102A100009F45FC08933910509F10895833E91055A
:102A2000D9F138F4803E910529F1823E910579F182
:102A30000895863E9105D9F1873E910509F43EC07F
:102A4000843E910541F52091810321FF24C08091AE
:102A5000800384FD19C087EE90E0089520918003E3
:102A6000237009F05AC02091810323FF14C089E22A
:102A700090E008952091800320FD38C030918103BB
:102A800030FF09C024FF43C090E080E0089520910A
:102A9000800322FDF7CF08952091800322FD3AC0E4
:102AA0003091810330FD39C024FFF5CFEDCF209167
:102AB000800323FFF0CF24FDE7CFCDCF209180030B
:102AC00023FD2EC03091810331FFEECF84EE90E0E4
:102AD00008952091800325FFDECFC9CF2091800388
:102AE00025FD21C02091810323FFD5CF89E390E00C
:102AF000D2CF2091800326FFCECF8AE290E00895C6
:102B00002091800326FFC7CF81E390E0089583EEF4
:102B100090E0089582EE90E0089580EE90E00895B0
:102B200086EE90E0089585E390E00895909180030B
:102B300092FF10C041E0282F2471243009F040E0BA
:102B400031E0282F2871283009F030E0431711F0C8
:102B50002CE0822793FF10C041E0282F24712431FC
:102B600009F040E031E0282F2871283109F030E0E9
:102B7000431711F02CE082273091810330FF10C001
:102B800051E0282F2171213009F050E041E0282F39
:102B90002871283009F040E0541711F029E082270D
:102BA00031FF10C041E0282F2171213109F040E0B0
:102BB00031E0282F2871283109F030E0431711F057
:102BC00029E0822794FD877E089508950E944A1285
:102BD000811102C00E94EA120E94551280931D03C7
:102BE0000E945F1290938103809380030E94E515F9
:102BF0000E945A1290E00E940F0D8091B2029091B3
:102C0000B3020E94300D089508950E94041608959D
:102C100008950E9408160895E82FF0E0E757FC4F4A
:102C200080810895B0E0A0E0E8E1F6E10C94ED2E9B
:102C300085E592E00E94FE0689E8E82E83E0F82E02
:102C4000D0E0C0E090E5C92E92E0D92E08E412E071
:102C5000DF93CF93DF92CF920E9497078DE492E0AB
:102C60000E94FE06F70181917F010E94C7081F9212
:102C70008F931F930F930E94970786E492E00E9420
:102C8000FE0621968DB79EB708960FB6F8949EBFA4
:102C90000FBE8DBFC730D105D9F6CDB7DEB7E8E09E
:102CA0000C94092F80EA8A95F1F7089500C00895E1
:102CB0000E9452160895F894E82FE295EF70F0E024
:102CC00031A1282F2F7081E090E001C0880F2A9554
:102CD000EAF7982F9095932391A392A1892B82A331
:102CE000789408950F931F93CF93DF93CCE9D1E0AD
:102CF00089918F3F11F00E945B1681E0C33AD8079B
:102D0000B9F7C6E9D1E00CE911E089918F3F11F0E4
:102D10000E945B160C171D07C1F7DF91CF911F9121
:102D20000F910895B0E0A0E0E8E9F6E10C94ED2EF3
:102D3000EC01D62E062F10E0C80184569E4F7C0170
:102D4000FC0180818F3F09F444C0F894E82FE2959C
:102D5000EF70F0E091A18F7021E030E001C0220F10
:102D60008A95EAF7892F822B81A382A120952823B7
:102D700022A378940E945616E6E9F1E031E0C12CD6
:102D800021912F3F59F1A22FA295AF70B0E09096FC
:102D90008C9190E02F7002C0959587952A95E2F767
:102DA00080FD1CC0832FC82A330F81E0EC39F8075F
:102DB00039F7F70180818F3F11F00E945B1661E0C7
:102DC000C11001C060E08D2D0E945816C00FD11FA8
:102DD000C882CDB7DEB7E8E00C94092F80E0E3CFDE
:102DE0000E94721687E0E9E8F3E0DF01982F1D9258
:102DF0009A95E9F7E2E8F3E0DF011D928A95E9F799
:102E000087E00E9441170E9405160895A7E0B0E0F0
:102E1000ECE0F7E10C94F02E8E010F5F1F4F87E07E
:102E2000F80111928A95E9F7F12C6F2DC8010E94E3
:102E30009216F394F7E0FF12F8CF47E050E0B801A4
:102E400082E893E00E94B92F21E0009709F420E086
:102E5000892B41F087E0F801A2E8B3E001900D92E0
:102E60008A95E1F747E069E873E082E893E00E9421
:102E70004217182F0E940916812F2796E5E00C941F
:102E80000C2F0895B0E0A0E0E8E4F7E10C94ED2EFB
:102E90006C017B01042FC22F222379F081E0809303
:102EA00020030E94A02690931F0380931E0380E0BE
:102EB000CDB7DEB7E8E00C94092FD0912003DD23D5
:102EC000B1F380911E0390911F030E94B8260597CD
:102ED00070F310E0A801B601C7010E94B92F892B39
:102EE00031F0A801B601C7010E94C62FCD2F109264
:102EF00020038C2FDDCF0E9418290E9450130E94BE
:102F0000252908950E942A290E945B130E944C29BA
:102F100008950E9439260E94FE280E9433130E94C1
:102F20007B170E9482170E944613FBCF9093930257
:102F3000809392020895EF92FF920F931F93CF9385
:102F4000DF93EB01E82FD1110EC0442321F0F0E014
:102F5000E151F94FE4916E2F7E2F8E2FCDB7DEB762
:102F6000E6E00C940B2F0D2F10E0282F30E04423C7
:102F700029F02151394FF901249130E0F6E0CF9F3B
:102F8000C0011124EFEFF0E0BF010E94622EAB01FF
:102F90008C2F90E0880F991FA5E5A49FB001A59FF5
:102FA000700D1124861B970B982F990F980FBF0156
:102FB000601B710B629FD001639FB00D729FB00DBB
:102FC00011248B2F9D9FB0011124672F7727EF01CC
:102FD000C61BD70BBE01629FE001639FD00D729F9D
:102FE000D00D11247F01E91AF108E09EB001E19EA5
:102FF000700DF09E700D1124672F7727E61BF70BDD
:10300000E29F8001E39F100DF29F100D1124E12F2C
:10301000722F4230510599F048F44115510569F07D
:103020004130510581F0EB2F8D2F07C04430510501
:1030300069F080F046305105B1F76E2F8FCFE22F47
:103040007B2F812FFACFE22F7D2FF7CFEB2F822F0F
:10305000712FF3CF7B2F822FED2FEFCF41E00E9416
:103060009B17089508950E942E180895CF93DF931B
:10307000762FE901682F842F0E94331879836883A3
:103080008A83DF91CF91089580919003982F9C7F40
:1030900029F4837084608093900308958C3AE8F358
:1030A0008370886AF8CFB0E0A0E0E9E5F8E10C941D
:1030B000ED2E88E090E00E94D72F6B017C0184E226
:1030C00090E00E94CF2F282F30E040E050E060E0F9
:1030D00070E080E090E000E20E941A2FB22FA32F50
:1030E000F42FE52FD62FC72F97018601BC29A12BDE
:1030F000FE295E2F532B2B2F3A2F4F2F6D2F7C2F16
:10310000CDB7DEB7E8E00C94092FB0E0A0E0EBE823
:10311000F8E10C94E92E49015A016B017C010E94EF
:1031200044188401A4016A2D7B2D88E090E00E9460
:10313000053094014A2D5B2DB601C70100E20E94C3
:10314000352F622F84E290E00E94F32FCDB7DEB7D7
:10315000ECE00C94052FE0E9F3E085E08083118238
:103160008FEF828383831482758125E030E04FEFF7
:103170005FEF60E0868197810E94851808958091B5
:103180001D0380FF8BC08CEB95E09F938F930E9473
:10319000970780911D030F900F9080FF7FC0809153
:1031A000900381701F928F938FE995E09F938F9387
:1031B0000E94970780911D030F900F900F900F9022
:1031C00080FF6CC080919003869581701F928F93D1
:1031D0008FE795E09F938F930E94970780911D033F
:1031E0000F900F900F900F9080FF58C08091900328
:1031F000869586951F928F9384E695E09F938F9393
:103200000E94970780911D030F900F900F900F90D1
:1032100080FF44C0809191031F928F938AE495E0D0
:103220009F938F930E94970780911D030F900F909B
:103230000F900F9080FF32C0809192031F928F9366
:1032400080E395E09F938F930E94970780911D03E1
:103250000F900F900F900F9080FF20C080919303EC
:103260001F928F9386E195E09F938F930E9497071B
:1032700080911D030F900F900F900F9080FF0EC054
:10328000809194031F928F938AEF94E09F938F9382
:103290000E9497070F900F900F900F9008958091C4
:1032A000900380FF03C086958695089580E0089579
:1032B00090919403933018F49F5F90939403882324
:1032C00091F020919003309191034091920350919D
:1032D000930360919403709195038091960390916C
:1032E00097030E948518089581E00E945819089557
:1032F00090919403992319F091509093940388230B
:1033000091F020919003309191034091920350915C
:10331000930360919403709195038091960390912B
:1033200097030E948518089581E00E9478190895F6
:1033300070E00E944221089560910A0180919003FB
:1033400080FF0BC08091090123E0829FC0011124FE
:1033500088569C4F0E949819089580910B01909176
:103360000C0123E0829FF0011124E856FC4F8917DD
:1033700048F71182108212828F5F3396F8CF9091B6
:10338000900390FF0EC090910B0120910C0133E04F
:10339000939FF0011124E856FC4F921718F00E94F9
:1033A0009C1908958183608342839F5F3396F5CF94
:1033B000A3E0B0E0EEEDF9E10C94F32E90919003D0
:1033C00090FF0AC09E012F5F3F4F0E9436184B812D
:1033D00069818A810E94BF192396E2E00C940F2F25
:1033E000CF93DF93EC01EC81F0E0E651FA4F44918A
:1033F000E0E9F3E0628181810E94D8198C818F5FBE
:103400008C83DF91CF910895CF93DF93EC01E0E9B6
:10341000F3E0438162818C810E94D8198C818F5F97
:103420008C83DF91CF910895A3E0B0E0EAE1FAE167
:103430000C94F12E8C018091210381110AC09E0110
:103440002F5F3F4F4FEF6FEF0E9436188A818093B6
:103450002103F8016481613069F08091210340E02B
:10346000662361F040E0623011F44091210380E076
:1034700060E004C06091210340E080E00E94BF1939
:10348000F801848190E0019663E070E00E94762E5E
:1034900084832396E4E00C940D2FA3E0B0E0E3E5F1
:1034A000FAE10C94E62E082FE62EF42EC22E90910F
:1034B000900390FF4BC0E92FE695E695AE2FB0E064
:1034C000AD55BE4F8C91809364039C7F943009F07E
:1034D00041C09E012F5F3F4F802F0E9436184B81C5
:1034E00069818A810E94BF1900939103E09292033F
:1034F000F0929303CC2009F48AC02091900360914C
:10350000940370919503302FA701809196039091B9
:1035100097030E94851880911D0380FF17C080913A
:1035200093031F928F93809192031F928F938091A8
:1035300091031F928F938DEB92E09F938F930E9444
:1035400097070FB6F894DEBF0FBECDBF2396EFE00E
:103550000C94022F823019F4F0909303C5CF86307B
:1035600019F400919103C0CF8930D9F3893109F062
:10357000BBCFE9518E2F8170782E8E2F8095817070
:10358000D82EE695F0E0E651F94F1491612C92EEB9
:10359000A92E92E0B92E60910D01661618F00E94D6
:1035A0009C19A2CF619EC001112470E00E94622E7E
:1035B000502E71102AC0560E862C912C80911D031E
:1035C00080FF11C01F921F931F92DF921F925F9284
:1035D0001F926F92BF92AF920E9497070FB6F89416
:1035E000DEBF0FBECDBF20910B01820E911C940156
:1035F000220F331F280D391D28563C4F4F2D6E2D9D
:10360000852D0E9436186394C6CF561AD5CF809167
:103610001D0380FF9BCF1F92FF921F92EF921F927C
:103620000F9386E992E089CFE0E9F3E09181282FBA
:103630004381628180E1890F0E944D1A089581E0E3
:103640000E94141B0895E0E9F3E09181282F438143
:10365000628180EF890F0E944D1A089581E00E94D7
:10366000231B0895E0E9F3E0628120E1620F08F492
:103670006FEF282F438181810E944D1A089581E0C8
:103680000E94321B0895E0E9F3E0628120E1621BB1
:1036900008F460E0282F438181810E944D1A08952B
:1036A00081E00E94431B0895E0E9F3E0438120E1BB
:1036B000420F08F44FEF282F628181810E944D1A3A
:1036C000089581E00E94541B0895E0E9F3E04381EE
:1036D00020E1421B08F440E0282F628181810E9492
:1036E0004D1A089581E00E94651B089520E00E9414
:1036F0004D1A0895EF92FF921F93CF93DF93EC0141
:1037000010E0EE24EA94F12C60910D01161770F090
:103710000E949C199A818C8190FF27C08F5F8C83B7
:10372000DF91CF911F91FF90EF90089520910B01B1
:10373000422F410F5527551FCA019A01220F331FEF
:10374000280F391F28563C4F70E0C7010E94762E83
:10375000962F8C814091930360919203199F800D65
:1037600011240E9436181F5FCFCF8150D8CFB0E010
:10377000A0E0EDEBFBE10C94EB2EFC0182810FEF5E
:1037800080FF01E010E04BE0A42E80910D0118179E
:1037900098F00E949C1980912303013009F04FC0DA
:1037A000811102C080910D01815080932303CDB718
:1037B000DEB7EAE00C94072FC0910B01C12ED12C8B
:1037C000CC0DDD2DD11DCE01880F991FC80FD91F3B
:1037D000C856DC4F198218821A8234E0E32EF12C8D
:1037E000B12C809123038B0D8C301CF16A2D0E942B
:1037F000542E892F082E000C990BC816D90691F467
:10380000809193038E9DA0018F9D500D112455959D
:103810004795559547959E0160919203809191033C
:103820000E943618B00EF1E0EF1AF108D1F61F5FD2
:10383000ACCF87FFDFCF90910D01890FDBCF90E0F8
:10384000019660910D0170E00E94762EAECF0F932D
:103850001F93CF93DF9380910B0190910C0123E094
:10386000829FF0011124E856FC4F891740F1C0E017
:10387000D3E060910D01C61740F10E949C19209180
:10388000070180912203820F809322039091080107
:10389000920F90930801191654F4082E000C990BFE
:1038A00040910D014150550B841795071CF021954F
:1038B00020930701DF91CF911F910F9108951182FD
:1038C000108212828F5F3396D0CF0C2F10E070E001
:1038D000C8010E94762E20910B01820F482F50E0E4
:1038E00020912203022E000C330B02171307BCF0A9
:1038F00020910801022E000C330B201731077CF0B9
:103900008D9F9001112428563C4F40919303609164
:103910009203809191030E943618CF5FAACFFA01DB
:10392000EE0FFF1FE40FF51FE856FC4F11821082C7
:103930001282F3CFB0E0A0E0E0EAFCE10C94E92EC3
:10394000EC014C81042F10E09801D8010E94BA2E9E
:103950009B01AC010E94D02E4B015C01E0E2F0E043
:10396000E01BF10BA5E5B0E0AC019B010E94D02E5D
:103970006B017C019F01DF010E94B22E9B01AC0113
:103980000E94DB2E9B01AC01280D391D4A1D5B1DD9
:10399000C701B6010E948A2EF22E822F90E039E2F2
:1039A0003F1520F143E0249F900111243595279580
:1039B000122F109500E085E5E82EEF1880910D019B
:1039C000081718F10E949C199C8181E0992319F035
:1039D000903219F48FEF8093060180910601890FD0
:1039E0008C83CDB7DEB7ECE00C94052F25E530E0F5
:1039F000B901681B790B9B01220F331F260F371F5C
:103A000037FFD4CF2F5F3F4FD1CF8E2D01FD8F2DAC
:103A100020910B01622F600F7727771F9B01220FE8
:103A2000331F260F371F28563C4F412F60919203BA
:103A30000E9436180F5FC2CF0F931F93CF93DF936F
:103A4000EC0110E000E090910D019017110609F0D3
:103A50006CF40E949C198C8190E0019681709927EA
:103A60008C83DF91CF911F910F91089520910B01CD
:103A7000A801420F511D9A01220F331F240F351F39
:103A800028563C4F4C81609192038091910396950A
:103A90009017110651F04CF0442349F040919303E4
:103AA0000E9436180F5F1F4FCECF4423B9F340E07A
:103AB000F7CFB0E0A0E0EFE5FDE10C94E52EFC01CE
:103AC0006280448081E08483EAEEF5E07490E9E668
:103AD000F6E0E491C0919303C695C158D0E0CC0FB5
:103AE000DD1FCD2FDD27812C75E0972EAA24AA9407
:103AF000B12C55245A94E719EE2EF12C80910D012A
:103B0000881638F00E949C19CDB7DEB7E0E10C941E
:103B1000012FC82CD12C82E0861568F09C9CF00106
:103B20009D9CF00D1124EC5DFC4F809191038083EE
:103B3000809192038183411023C09C9CF0019D9C45
:103B4000F00D1124EC5DFC4F1382128220910B01C9
:103B5000C601820F911D9C01220F331F280F391FB0
:103B600028563C4F9C9CF0019D9CF00D1124EC5D6F
:103B7000FC4F4281618180810E9436188394BECFC0
:103B80009C9C80019D9C100D11240C5D1C4FF80124
:103B900083818823F1F081508383859DC0011124A6
:103BA000648170E00E94622EFB01FF27E651FA4F0C
:103BB0008491E82FE719E59DC0011124B7010E9407
:103BC000622E80919303689FB0011124F8017283E3
:103BD000BDCF0E949C2FB5010E94762E8C179D07A9
:103BE0000CF0B4CFF2E0F61598F40E949C2FB501CA
:103BF0000E94762EF80180830E949C2F20919203D0
:103C00002695622F70E00E94762E280FF8012183FE
:103C10009C9CF0019D9CF00D1124EC5DFC4F1282E8
:103C200080919303893C58F088EC9C9CF0019D9C0A
:103C3000F00D1124EC5DFC4F8483838387CF8431A6
:103C4000A0F784E1F2CF609190036695669570E0ED
:103C50004BE050E08EE091E00E94AC2F892B19F4EC
:103C600081E0809365030E94A02690935C0380937B
:103C70005B0380911D0380FF08C08DE792E09F9356
:103C80008F930E9497070F900F90089510926503ED
:103C900080911D0380FF08C084E692E09F938F937C
:103CA0000E9497070F900F9008959091900390FFB6
:103CB00049C09370811147C0946090939003209104
:103CC0009003662309F447C0309191034091920319
:103CD00050919303609194037091950380919603A2
:103CE000909197030E94851880911D0380FF10C05A
:103CF00080919003869586951F928F9380E494E03F
:103D00009F938F930E9497070F900F900F900F90A3
:103D1000609190036695669570E04BE050E08EE010
:103D200091E00E94AC2F892B09F10E94461E81E090
:103D300080935E034091930360919203809191037D
:103D40000E94761B08958B3210F0986AB6CF880FC8
:103D5000880F982BB2CF80911D0380FFD9CF269575
:103D600026951F922F9382E294E0CACF0E94231ED1
:103D7000DECF682F909190039695969581E0890FFC
:103D80008B3208F081E00E94551E089581E00E9468
:103D9000B91E0895682F90919003969596958FEF90
:103DA000890F09F48AE20E94551E089581E00E945D
:103DB000CA1E089561E00E94551E089580919003E7
:103DC00081608093900380911D0380FF0DC01F923E
:103DD00081E08F9384EB93E09F938F930E949707EA
:103DE0000F900F900F900F9080919003869586957D
:103DF0000E94DA1E089560E00E94551E0895809189
:103E00006303811171C080911D0380FF14C083EE94
:103E100094E09F938F930E94970780911D030F90CA
:103E20000F9080FF08C08DEC94E09F938F930E94C9
:103E300097070F900F900E944A12811110C0809135
:103E40001D0380FF08C085EA94E09F938F930E9432
:103E500097070F900F900E94EA120E94AB180E94E1
:103E600053182093900330939103409392035093FF
:103E700093036093940370939503809396039093B8
